:1000000012C02AC029C028C032C026C025C024C0C2
:1000100023C022C021C020C01FC01EC01DC01CC0E4
:100020001BC01AC019C011241FBECFEDCDBF10E0F8
:10003000A0E6B0E0EAEEF0E002C005900D92A8372D
:10004000B107D9F710E0A8E7B0E001C01D92A937C9
:10005000B107E1F73BD047C0D3CF20ED37E004C074
:10006000F9013197F1F701970097D1F708951F92A1
:100070000F920FB60F9211242F933F938F939F935C
:10008000EF93FF938091780090E020916000309191
:1000900061008217930714F0109278008091780025
:1000A000E82FF0E0EE0FFF1FEE59FF4F908198BB55
:1000B0008F5F80937800FF91EF919F918F913F9197
:1000C0002F910F900FBE0F901F9018958FEF87BB49
:1000D00089E08EBD80E197E29BBD8ABD89B78064CF
:1000E00089BF7894FFCFF894FFCF0B0000000E007B
:1000F0003F007E00FC007E003F000E00000000007C
:100100000000FFFFFFFFFFFFFFFFFFFFFFFFFFFFFD
:10011000FFFFFFFFFFFFFFFFFFFFFFFFFFFFFFFFEF
:10012000FFFFFFFFFFFFFFFFFFFFFFFFFFFFFFFFDF
:10013000FFFFFFFFFFFFFFFFFFFFFFFFFFFFFFFFCF
:10014000FFFFFFFFFFFFFFFFFFFFFFFFFFFFFFFFBF
:00000001FF
